:03000B00020C6F75
:0300230002074889
:03002B0002167743
:10060000021829D2B57407120808743312080812A8
:100610000844300CFDC2B575260022D2B57407120D
:1006200008087433120808120844158115811581D1
:10063000300CFDC2B575260022B4300100400FB465
:100640003A004011B441004005B447004004C200E4
:100650008008C39407C39430D20022540FB40A0018
:10066000400224072430227583017582007400F053
:100670000582E582B4FFF6220102040810204080C2
:10068000C0F0E0D1393000028004C200C11BC4F5C3
:10069000F00582E0D1393000028004C200C11B4560
:1006A000F00582D0F022C083C082C0E0C2969015CF
:1006B0005574AAF0900AAA7455F090155574A0F0DC
:1006C000D0E0D082D08322C083C082C0E0C29690A6
:1006D000555574AAF0902AAA7455F090555574A0F7
:1006E000F0D0E0D082D08322C28CD2B5C000F81204
:1006F000070DC297D1C7F0D296F8E0B500FBD297AC
:10070000D000300CFDC2B5752600D28C22C0E0C0EE
:1007100082C0839006A6E493F0A3E583B407F7E5CF
:1007200082B40DF2D083D082D0E0229005FAE49317
:10073000C235B48002D2350582E493C234B480025B
:10074000D23422D20E0207FD209807D20CC29902A1
:100750000807C298C083C082C0E0C0F0C0D0E5994D
:1007600020D0E0C2E7B42109C208D209D20A0207A8
:10077000FD300B030207FDBF00030207C52008453B
:10078000200D29200911200A030207FDB40D6EC2B5
:100790000A7508000207FDC209D13930005F8FF0E9
:1007A000C453F0F0B5F056D20D0207FDC20DD13999
:1007B00030004A8FF053F00FB5F042D20874D9756B
:1007C00008000207D6B4080EE508B400030207FDCE
:1007D00014F5080207FD900100850882B46100400D
:1007E00007B47B005002C2E5F00582858208B40D93
:1007F0000CC20AD20B150885081E750800D0D0D08F
:10080000F0D0E0D082D08332300CFDC20CA2D09266
:10081000E7F599C2E7C082C083852682758302F01E
:10082000A3858226D083D08222C0E0C082C083907C
:100830000000A3E583B410FAE582B400F5D083D0BC
:1008400082D0E022C0E0740D1108D0E022D2B5C001
:10085000E0C082C083E493B4000F300CFDC2B575D4
:100860002600D083D082D0E022B2B21108A3015575
:10087000C0E0C0E0C412065B1108D0E012065B11B4
:1008800008D0E022C083C082900100D2B5E0B40D50
:100890000F1108D082D083300CFDC2B5752600221E
:1008A00011080582018DC083C082900200D2B5E09C
:1008B000B40D0F1108D082D083300CFDC2B575265F
:1008C00000221108A301AF900000D2B575F080207E
:1008D000340375F020B2B2740093117074201108C3
:1008E000A3E583B5F0EFE582B4FFEA744411087420
:1008F0004F1108744E110874451108740D11083019
:100900000CFDC2B575260022D2B5743F110874459E
:10091000110874721108747211087453110874501C
:100920001108740D1108300CFDC2B5752600229017
:100930000101E0B452D20582E0B44FCC0582E0B4AC
:1009400047C60582E0B452C00582E0B441BA0582D0
:10095000E0B44DB40582E0B43DAEE4C0E0C0E022B6
:10096000D2B5743D110874501108746F1108746485
:100970001108742011089018E47400931170FF900E
:1009800016BA114D300CFDC2B5752600223F4572D6
:10099000723820496E76616C69642042617564200A
:1009A000526174650D00D2B590098D114D300CFD6A
:1009B000C2B5752600223F4572723720496E7661B6
:1009C0006C6964204261756420436F6D6D616E6473
:1009D0000D00D2B59009B6114D300CFDC2B575268B
:1009E0000022900101E0B441E90582E0B455E3053D
:1009F00082E0B444DD0582E0B43DD70582E0F5F045
:100A00000582E0B5F0CC0582E0B5F0C6B430004018
:100A1000C1B4380050BC120639F954079005FF12D2
:100A200006E8D2B5743D1108743A110874421108F1
:100A3000746111087475110874641108743A11080E
:100A4000E91170740D1108300CFDC2B57526001245
:100A500005FC223F4572723620496E76616C6964EE
:100A600020416464722052616E67650D00D2B590BA
:100A70000A53114D300CFDC2B575260022900104B9
:100A8000E01206393000028005C200020603C4F5F8
:100A9000F00582E01206393000028005C20002062D
:100AA0000345F0F99018E41206E8D2B5743D110838
:100AB000743A110874501108746F110874641108A5
:100AC00074231108E9FF1170740D1108300CFDC278
:100AD000B5752600D297000000C208223F45727209
:100AE0003520536574506F6441646472657373207C
:100AF0004572726F720D00900100E0B44603020B64
:100B00007DB44903020E0EB44F03020EC2B4530368
:100B10000213B9B443030210F2B45203021162B4D7
:100B2000420221E2B44D0302127BB456030212C208
:100B3000B44E030212E2B459030212F7B454030292
:100B40001372B45003020B8AB448022160B4440308
:100B5000020BBBB45703020BC6B43F0302159FB48C
:100B6000D9030212F7616790172E114D118422D21A
:100B7000B51144300CFDC2B5752600222290010348
:100B8000E0B42C030211D702155B0582E0B4521ABF
:100B9000900107E0B43F080582E0B40D1601C7B428
:100BA0003D110582E0B40D0B212F900106E0B40D3C
:100BB00002417D9016F6114D118422A3E0B40D037D
:100BC0000210C20214C3900101E0B43D0A90010674
:100BD000E0B40D09020C1DB43F03020BEFD2B59037
:100BE00016F6114D1184300CFDC2B575260022D2C7
:100BF000B57459A2044002744E1108E5131170E552
:100C000012117012180E742C1108E5131170E512F0
:100C100011701144300CFDC2B575260022900102FE
:100C2000120680F513F5CB120680F512F5CAC28CB8
:100C30009018E21206E8E5139018E2A31206E8D233
:100C40008CD2B5E5131170E51211701144300CFD12
:100C5000C2B575260022C0E0C000C3332432F88636
:100C600083088682A3A68218A683D000D0E022B291
:100C7000B2C0E0C083C082C0F0C000C001C002C0EA
:100C800003C004C005C0D0C28C9018E5E493F58C75
:100C9000E4A393F58AD28C908000E090B000E52D1B
:100CA000550DF07583C0E52E550EF07583D0E52FF8
:100CB000550FF07583B0E0F51B7583C0E0F51C752A
:100CC00083D0E0F51D7900B90803020D1E90067867
:100CD000E993FBE50D5BB40020E51B5BFDE5275BBD
:100CE0006DB50312E5095BB50303750C01E52A5BDD
:100CF000B50503E99156020D1AE9C3332432F8E62B
:100D0000B40003020D1A14F6B4000FE52D6BF52D97
:100D1000E9C333042432F8E618F6050181C7851BC0
:100D2000277900B90803020D80900678E993FBE566
:100D30000E5BB40022E51C5BFDE5285B6DB503147A
:100D4000E50A5BB50303750C01E52B5BB50505E909
:100D500024089156020D7CE9C33324322410F8E6AE
:100D6000B40003020D7C14F6B40011E52E6BF52ED1
:100D7000E9C3330424322410F8E618F60501A12350
:100D8000851C287900B90803020DE2900678E993E2
:100D9000FBE50F5BB40022E51D5BFDE5295B6DB54E
:100DA0000314E50B5BB50303750C01E52C5BB5057E
:100DB00005E924109156020DDEE9C33324322420C4
:100DC000F8E6B40003020DDE14F6B40011E52F6B53
:100DD000F52FE9C3330424322420F8E618F6050180
:100DE000A185851D29D0D0D005D004D003D002D054
:100DF00001D000D0F0D082D083D0E0322432F8A6E7
:100E0000F02274322430F8187600B832FA229001B9
:100E100001E0B44C09E51BD2B51170020EAFB44D20
:100E200009E51CD2B51170020EAFB44809E51DD218
:100E3000B51170020EAFB40D11E51DD2B51170E5FC
:100E40001C1170E51B1170020EAF900103E0B40D90
:100E500069900101E01206393000028005C20002EB
:100E60000603C4F5F00582E0120639300002800561
:100E7000C20002060345F0B418005029781B20E494
:100E80000620E304020E89080886019006785407BC
:100E900093FBE95BB400057430020E9E7431D2B549
:100EA0001108020EAFD2B57407110874341108117D
:100EB00044300CFDC2B5752600229016F6114D1176
:100EC0008422900101E0B44C29A3E01206393000DD
:100ED000028005C200020603C4F5F00582E0120696
:100EE000393000028005C20002060345F0F52D02EC
:100EF00010A1B44D29A3E01206393000028005C2CA
:100F000000020603C4F5F00582E012063930000243
:100F10008005C20002060345F0F52E0210A1B44878
:100F200029A3E01206393000028005C20002060340
:100F3000C4F5F00582E01206393000028005C200D7
:100F400002060345F0F52F0210A1900107E0B40D51
:100F500074900101E01206393000028005C20002DF
:100F60000603C4F5F0A3E01206393000028005C282
:100F70000002060345F0F52FA3E012063930000207
:100F80008005C200020603C4F5F0A3E01206393062
:100F900000028005C20002060345F0F52EA3E01210
:100FA00006393000028005C200020603C4F5F0A332
:100FB000E01206393000028005C20002060345F047
:100FC000F52D0210A1900102E0B42D0AA3AC82AD70
:100FD000837900020FE0B42B1CA3AC82AD837901AE
:100FE000900101E01206393000028005C2000206BD
:100FF00003FA021037900103E0B42D0AA3AC82ADCE
:10100000837900021010B42B577901A3AC82AD8311
:10101000900101E01206393000028005C20002068C
:1010200003C4F5F00582E01206393000028005C2E3
:101030000002060345F0FA782D20E40620E30402BE
:101040001044080890067854079386F0B9010645C5
:10105000F0F6021059F455F0F68C828D830210637D
:101060000210AFE0B40D030210A1D2B51206393060
:1010700000028005C200020603C4F5F0A3E01206D8
:10108000393000028005C20002060345F0F5F0EA9F
:10109000D2B5C323120DFC75F000EAC32304120D70
:1010A000FCD2B5120844300CFDC2B5752600229062
:1010B00016F612084D12088422900100744FF002B7
:1010C0000AF7C28CD2B5900300B2B2E0120870A346
:1010D000E0120870A3E0120870A37420120808E55B
:1010E00083B41FE5120844300CFDC2B5752600D24A
:1010F0008C22900103E0B40D5F900101E0120639EB
:101100003000028005C200020603C4F5F00582E04B
:101110001206393000028005C20002060345F0B411
:101120001800501CC3332432F8E6D2B512087008F8
:10113000E6120870120844300CFDC2B57526002274
:10114000D2B5740712080874341208081208443023
:101150000CFDC2B5752600229016F612084D120835
:101160008422900103E0B40D18900101120680B4AE
:1011700018005037C3332432F87600087600021185
:101180009D900101E0B4413B0582E0B44C350582FD
:10119000E0B44C2F0582E0B40D29120E02D2B51234
:1011A0000844300CFDC2B575260022D2B574071272
:1011B00008087434120808120844300CFDC2B575D2
:1011C0002600229016F612084D120884229016F678
:1011D00012084D12088422900106E0B40DEF900130
:1011E00001E01206393000028005C200020603C485
:1011F000F5F00582E01206393000028005C20002D7
:10120000060345F0FD780D20E40620E304021212E7
:10121000080823F9900104E0120639300002800525
:10122000C200020603C4F5F00582E0120639300060
:10123000028005C20002060345F0F5F0ED54079068
:10124000067893FBE65BB40003021263E92432F8EC
:10125000E5F0F608F6D2B5120844300CFDC2B575BB
:10126000260022D2B5740712080874341208081236
:101270000844300CFDC2B575260022900104E0B48C
:101280000D28900101E0B44C09A3120680F50D026F
:1012900012B4B44D09A3120680F50E0212B4B4487C
:1012A00009A3120680F50F0212B49016F612084D2B
:1012B00012088422D2B5120844300CFDC2B575263E
:1012C0000022900101E0B40D0F9016B412084D30C9
:1012D0000CFDC2B5752600229016F612084D1208B4
:1012E0008422900101E0B40D041208A6229016F6A3
:1012F00012084D12088422900101E0B40D2CD2B5E1
:10130000E50CB40011744E120808120844300CFDAC
:10131000C2B5752600227459750C0012080812080F
:1013200044300CFDC2B5752600229016F612084D09
:1013300012088422900101E0B40D30D2B5EF1208FA
:1013400070E50CB40011744E120808120844300CF9
:10135000FDC2B5752600227459750C0012080812DA
:101360000844300CFDC2B57526002290176412089F
:101370004D22900104E0B40D28900101E0B44C0925
:10138000A3120680F5090213ABB44D09A31206801F
:10139000F50A0213ABB44809A3120680F50B021339
:1013A000AB9016F612084D12088422D2B5120844EA
:1013B000300CFDC2B575260022900102E0B40D2369
:1013C000900101E0B43F3F9018E5E493D2B51208D4
:1013D00070E4A393120870120844300CFDC2B57576
:1013E000260022900105E0B40D07900101E00214EF
:1013F00009900106E0B40D0E900101E0B44307FD31
:101400000582E00214090214B91206393000028084
:1014100005C200020603C4F5F00582E01206393069
:1014200000028005C20002060345F0F80582E012C2
:1014300006393000028005C200020603C4F5F0053B
:1014400082E01206393000028005C2000206034520
:10145000F0F9F4F582E8F4F583A3AA83AB82E8B44B
:1014600003005003021470B4030CE9B49A00500650
:1014700078DC74008152C28CEA9018E51206E8EB21
:10148000A31206E8D28CD2B5EDB4431D793274189C
:10149000B2B2B7000709B700080214A577010980A6
:1014A000041977010909D5E0E7D28CD2B5120844B6
:1014B000300CFDC2B5752600229016F612084D12AA
:1014C000088422900102E0B42D0579000214D4B4FE
:1014D0002B177901900101E01206393000028005D6
:1014E000C200020603FA021521900103E0B42D05A3
:1014F00079000214FAB42B597901900101E0120627
:10150000393000028005C200020603C4F5F00582EE
:10151000E01206393000028005C20002060345F0E1
:10152000FA782A20E40620E30402152E0808900623
:101530007854079386F0B9010645F0F6021543F496
:1015400055F0F6D2B5120844300CFDC2B575260030
:10155000229016F612084D12088422900109E0B478
:101560000D331582E0B44C087A8012163902158FBB
:10157000B44D087A9012163902158FB448087AA033
:1015800012163902158FB4410C0215951215E3900D
:10159000030001C2229016F612084D120884229010
:1015A000179212084D900101E0B40D099017CA126C
:1015B000084D0215E2B431099017CA12084D021500
:1015C000E2B432099017CA12084D0215E2B4330989
:1015D0009017CA12084D0215E2B434D09017CA12FF
:1015E000084D22C083C082C0E0C001C003C004C057
:1015F00005C006900300B2B2908000E0FE7583C083
:10160000E0FD7583D0E0FC851183851082ECF0A3AA
:10161000EDF0A3EEF0A3858311858210E583B41F5E
:10162000D78911858210B2B2D006D005D004D0037C
:10163000D001D0E0D082D08322900300A9838A8396
:10164000758200E089838B82F0A3A983AB82B2B25A
:10165000B920EB8911858210221217D8D20490B0DC
:1016600000E52D550DF07583C0E52E550EF0758300
:10167000D0E52F550FF022B2B2C0E0C083C082C0C7
:1016800000C0D02004217400B51206B51303021661
:10169000A7151274FFB5120215137400B51208B520
:1016A0001305D1590216A7D0D0D000D082D083D054
:1016B000E0C2CF32332E31350D002C205244472D5D
:1016C000323420526576204234204669726D77614B
:1016D0007265205665723A332E31352041434345B9
:1016E0005320492F4F2050726F64756374732C2000
:1016F000496E632E0D004572726F722C20757365F2
:10170000203F20666F722073796E7461782C20639D
:101710006F6D6D616E64206E6F742066756C6C7990
:10172000207265636F676E697A65643A200045725E
:10173000726F722C20757365203F20666F72206374
:101740006F6D6D616E64206C6973742C20756E72A0
:1017500065636F676E697A656420636F6D6D616E36
:10176000643A20004572726F722C20416464726585
:10177000737320636F6D6D616E64206D757374207B
:101780006265204352207465726D696E6174656490
:101790000D00414343455320492F4F2050726F6441
:1017A000756374732C20496E632E20436F6D6D61D9
:1017B0006E64205265666572656E636520666F7241
:1017C000205244472D32340D0D0048656C70207254
:1017D000656D6F7665640D00C28C750D00750E0029
:1017E000750F007509FF750AFF750BFF752DFF75E5
:1017F0002EFF752FFF752AFF752BFF752CFF120E1C
:1018000002C204300CFDC2B5752600D28C22C0E0A5
:10181000C082C083C2049018E2E493F512E4A3935B
:10182000F513D083D082D0E022758162C0E07508C4
:1018300000D2AFD20C1205FC9018E5E493F58CE4CD
:10184000A393F58A1217D8C2CA75C80090DC008528
:1018500082CC8582CA8583CD8583CB9018E2E493C0
:10186000F513E4A393F5127400B51206B513030241
:101870001878C2BDD2ADD2CAD2BCC2B99018E47435
:101880000093FF900000C20B1206677510007511DF
:1018900003D235C234D28C300CFDC2B5752600D0CF
:1018A000E0B400030218A9D298D2A9B2B2300BFB5F
:1018B000200E0F120829120AF7110EC20B1206672A
:1018C00001ABD2B57407120808743912080812085F
:1018D00044300CFDC2B5752600C20EC20B1206675D
:0818E00001AB000000DC001167
:00000001FF
